:100000000C945C000C943D050C946A050C948400DF
:100010000C9484000C9484000C9484000C94840050
:100020000C9484000C9484000C9484000C94840040
:100030000C9484000C9484000C9484000C94840030
:100040000C9497050C9484000C94C9070C948400BC
:100050000C9484000C9484000C9484000C94840010
:100060000C9484000C948400000024272A000025AE
:10007000282B000023262904040404040404040299
:100080000202020202030303030303010204081035
:100090002040800102040810200102040810200002
:1000A0000000070002010000030406000000000039
:1000B00000000000F401290411241FBECFEFD4E09A
:1000C000DEBFCDBF11E0A0E0B1E0E2E2F1E102C0AD
:1000D00005900D92A433B107D9F712E0A4E3B1E083
:1000E00001C01D92A130B107E1F710E0C8EBD0E0EC
:1000F00004C02297FE010E948B08C43BD107C9F7B8
:100100000E9422040C948F080C940000FC011082C1
:100110008FEF81831382128282E2848386E9858352
:10012000178216820895EF92FF920F931F93CF9339
:10013000DF93EC019B0177FF03C020E030E005C0B6
:10014000653B710514F024EB30E02983EC806D8170
:1001500070E06E197109882777FD8095982F982F88
:10016000872F762F662730E040E050E00E94060897
:1001700024EB30E040E050E00E945A08FF2400E009
:1001800010E0102F0F2DFE2CEE24E20EF31E041FA4
:10019000151FC801B70120E430E040E050E00E94A4
:1001A0005A083B832A83DF91CF911F910F91FF90D3
:1001B000EF9008955F926F927F928F929F92AF928D
:1001C000BF92CF92DF92EF92FF920F931F93DF9334
:1001D000CF93CDB7DEB76DB67EB6ADB65EB60E9434
:1001E0000706209136013091370140913801509136
:1001F0003901621773078407950750F02C5E3F4F53
:100200004F4F5F4F621773078407950708F4AFC01D
:1002100060933601709337018093380190933901D0
:10022000E0913401F0913501BB2408C082819381B3
:10023000892B09F0B3940680F781E02D3097B1F750
:10024000BB2009F494C08B2D90E0880F991F2DB727
:100250003EB7281B390B0FB6F8943EBF0FBE2DBF1B
:10026000CDB6DEB60894C11CD11CA0913401B0916A
:10027000350120E013C012968D919C911397892B24
:1002800049F0E22FF0E0EE0FFF1FEC0DFD1DB183F2
:10029000A0832F5F16960D90BC91A02D109759F753
:1002A0002CC0812F90E07C01EE0CFF1CEC0CFD1C9F
:1002B000D7016D917C91FC013197EE0FFF1FEC0D82
:1002C000FD1D40815181DB0112962D913C911397C8
:1002D000DA0112968D919C9113972817390730F403
:1002E000D7014D935C937183608301E01F5F1B1501
:1002F000C0F2002311F410E011C011E000E0F7CFCC
:10030000E12FF0E0EE0FFF1FEC0DFD1D0190F081DD
:10031000E02D61E080810E940D071F5F1B1580F3B7
:10032000F6B4EE2400E010E08F2C99241EC0EE2DD0
:10033000F0E0EE0FFF1FEC0DFD1D0190F081E02DB0
:1003400022813381280D391D86B58F1510F4005098
:100350001F4FF82EC8018F0D911D28173907A0F7E0
:1003600060E080810E940D07E394EB1400F38A2D76
:10037000952D9C010FB6F8943EBF0FBE2DBF0FB652
:10038000F8947EBE0FBE6DBECF91DF911F910F918D
:10039000FF90EF90DF90CF90BF90AF909F908F90A5
:1003A0007F906F905F9008950F931F938C01FC01D5
:1003B00060838FEF81831382128280913401909148
:1003C000350197838683109335010093340160E0F3
:1003D00080810E940D0761E0F80180810E94EF0694
:1003E00081E01F910F9108958AE391E00E948600B9
:1003F00082E491E00E9486008AE491E00E948600F7
:100400000895BC0182E491E00E9493000895BC012C
:100410008AE391E00E94930008956BE570E08AE31F
:1004200091E00E9493006AE570E082E491E00E940E
:10043000930008950F931F938C010E940D0264EBAB
:1004400070E0601B710B8AE391E00E949300B80199
:1004500082E491E00E9493001F910F9108950F9301
:100460001F938C010E940D02B8018AE391E00E9463
:10047000930064EB70E0601B710B82E491E00E94DA
:1004800093001F910F910895EF92FF920F931F9386
:10049000CF93DF930E94DA008BE691E00E9437044D
:1004A000882309F48EC08BE691E00E943404809387
:1004B0005C01482F50E09A01207F307080915D01EF
:1004C00090915E012817390709F07BC0EA01CF70CF
:1004D000D070C330D10509F451C0C430D1054CF4FB
:1004E000C130D10539F1C230D105ECF5CD2B69F021
:1004F00068C0CD30D10509F45DC0CE30D10509F416
:100500005BC02C9709F05DC048C06DE570E08AE4DF
:1005100091E00E94930010926A011092690160E0DC
:1005200070E080911D010E94970684EB90E00E948C
:100530001A0247C084EB90E00E942F0284E690E00C
:100540009093680180936701D0936A01C093690119
:100550000E940706609363017093640180936501B4
:10056000909366012EC080E090E00E94070280E038
:1005700090E00E94010264EB70E00AC084EB90E01E
:100580000E94010284EB90E00E94070260E070E0AC
:100590008AE491E00E94930002C00E940D02109232
:1005A0006A011092690160E070E080911D010E9473
:1005B000970607C061E001C060E080911F010E94C2
:1005C0000D070E9407069B01AC0160935F017093C9
:1005D0006001809361019093620180916901909123
:1005E0006A01019709F053C0809163019091640101
:1005F000A0916501B0916601281B390B4A0B5B0B7A
:100600008091670190916801AA2797FDA095BA2F64
:10061000281739074A075B07A0F16FEF70E0809158
:100620001D010E949706E0905F01F090600100912B
:100630006101109162018091630190916401A09128
:100640006501B0916601A8019701281B390B4A0B7F
:100650005B0B8091670190916801880F991FAA2711
:1006600097FDA095BA2F281739074A075B0778F03E
:10067000E0926301F09264010093650110936601BA
:1006800006C060E070E080911D010E949706DF9136
:10069000CF911F910F91FF90EF90089540E855E2A0
:1006A00060E070E08BE691E00E943A0464E670E05E
:1006B00080E090E00E94150660E070E080911D01EE
:1006C0000E9497066091290170912A018AE391E0C6
:1006D0000E94D40160912B0170912C0182E491E081
:1006E0000E94D40160912101709122018AE491E07D
:1006F0000E94D4010E940D026DE570E08AE491E051
:100700000E94930061E080911B010E94EF0661E06E
:1007100080911D010E94EF0661E080911F010E94FF
:10072000EF0660E08EE00E94EF0660E08FE00E943E
:10073000EF0660E080E10E94EF0660E081E10E9448
:10074000EF0661E08EE00E940D0761E08FE00E94FD
:100750000D0761E080E10E940D0761E081E10E94E8
:100760000D07809152010E947906815092403CF021
:1007700081E090E0909355018093540104C0109261
:10078000550110925401809123010E9479068150F5
:1007900092403CF082E090E09093570180935601A4
:1007A00004C01092570110925601809125010E94B9
:1007B0007906815092403CF084E090E0909359019A
:1007C0008093580104C010925901109258018091F1
:1007D00027010E947906815092403CF088E090E029
:1007E00090935B0180935A0104C010925B011092B8
:1007F0005A018091560190915701209154013091F6
:100800005501820F931F2091580130915901820F99
:10081000931F20915A0130915B01820F931F909397
:100820005E0180935D0160E071E08BE691E00E94E3
:100830003F0460915D0170915E018BE691E00E9442
:100840002D0508950E943F060E944E030E94440217
:10085000FDCF82E391E090936C0180936B0108954A
:10086000862F0E94910708950E94AA0708950E946A
:1008700099070895CB01BA010E94580708950F9374
:100880001F93CF93DF938C01EB0109C02196D80110
:10089000ED91FC910190F081E02DC80109956881EE
:1008A0006623A1F7DF91CF911F910F9108950F93C8
:1008B0001F938C01DC01ED91FC910190F081E02D02
:1008C0006DE00995D801ED91FC910190F081E02D4A
:1008D0006AE0C80109951F910F9108952F923F92E8
:1008E0004F925F926F927F928F929F92AF92BF9240
:1008F000CF92DF92EF92FF920F931F93DF93CF93EC
:10090000CDB7DEB7A0970FB6F894DEBF0FBECDBF50
:100910001C016A017B01411551056105710549F40E
:10092000DC01ED91FC910190F081E02D60E30995EF
:1009300054C0882499245401422E552466247724D7
:1009400001E010E00C0F1D1F080D191DC701B601B5
:10095000A30192010E943808F80160830894811C69
:10096000911CA11CB11CC701B601A30192010E94F8
:100970003808C901DA016C017D01C114D104E10418
:10098000F104F1F681E0E82EF12CEC0EFD1EE80CEE
:10099000F91C3E010894611C711CD501C40101972A
:1009A000A109B1096C01C818D90814C0F601EE0DEF
:1009B000FF1D60816A3010F4605D01C0695CD10187
:1009C000ED91FC910190F081E02DC1010995089411
:1009D000E108F1086E147F0449F7A0960FB6F89469
:1009E000DEBF0FBECDBFCF91DF911F910F91FF9062
:1009F000EF90DF90CF90BF90AF909F908F907F90BF
:100A00006F905F904F903F902F900895EF92FF92DC
:100A10000F931F93CF93DF93EC017A018B0177FF44
:100A20000FC0E881F9810190F081E02D6DE2099518
:100A300010950095F094E094E11CF11C011D111D2E
:100A40002AE0B801A701CE010E946E04DF91CF9188
:100A50001F910F91FF90EF9008950F931F938C01BA
:100A6000AB01662757FD6095762F0E940605C801E9
:100A70000E9457041F910F9108951F920F920FB675
:100A80000F9211242F933F934F935F936F937F9314
:100A90008F939F93AF93BF93EF93FF9380916D01DB
:100AA00090916E01892B29F0E0916D01F0916E011A
:100AB0000995FF91EF91BF91AF919F918F917F9198
:100AC0006F915F914F913F912F910F900FBE0F90BB
:100AD0001F9018951F920F920FB60F9211242F930B
:100AE0003F934F935F936F937F938F939F93AF93B6
:100AF000BF93EF93FF9380916F0190917001892BC9
:100B000029F0E0916F01F09170010995FF91EF914B
:100B1000BF91AF919F918F917F916F915F914F9115
:100B20003F912F910F900FBE0F901F9018951F921D
:100B30000F920FB60F9211242F938F939F93AF9321
:100B4000BF938091710190917201A0917301B09156
:100B500074010196A11DB11D8093710190937201E2
:100B6000A0937301B0937401809175019091760107
:100B7000A0917701B09178018050904CAF4FBF4F5A
:100B80008093750190937601A0937701B0937801DB
:100B900027C08091750190917601A0917701B09165
:100BA000780180589E43A040B04080937501909397
:100BB0007601A0937701B0937801809179019091AB
:100BC0007A01A0917B01B0917C010196A11DB11D1C
:100BD0008093790190937A01A0937B01B0937C017B
:100BE0008091750190917601A0917701B091780183
:100BF00081589E43A040B04060F6BF91AF919F9155
:100C00008F912F910F900FBE0F901F9018958FB757
:100C1000F8942091790130917A0140917B015091B3
:100C20007C018FBFB901CA010895EF92FF920F9323
:100C30001F937B018C018FB7F894409179015091FB
:100C40007A0160917B0170917C018FBF2FB7F8947E
:100C50008091790190917A01A0917B01B0917C0102
:100C60002FBF841B950BA60BB70BE816F9060A07D6
:100C70001B0760F71F910F91FF90EF9008957894F4
:100C800084B5826084BD84B5816084BD85B5826091
:100C900085BD85B5816085BDEEE6F0E0808181602F
:100CA0008083E1E8F0E080818260808380818160E0
:100CB0008083E0E8F0E0808181608083E1EBF0E018
:100CC000808184608083E0EBF0E0808181608083BC
:100CD000EAE7F0E0808184608083808182608083A5
:100CE0008081816080838081806880831092C100D0
:100CF00008958F7090912D019295990F990F907C86
:100D0000982B90937C0080917A00806480937A0085
:100D100080917A0086FDFCCF209178004091790087
:100D2000942F80E030E0282B392BC90108951F93C0
:100D3000CF93DF93182FEB0161E00E94EF06E12FC4
:100D4000F0E0E156FF4F8491833051F480918000B0
:100D5000806880938000D0938900C09388003BC056
:100D6000843051F480918000806280938000D09321
:100D70008B00C0938A002FC0813039F4209729F16D
:100D800084B5806884BDC7BD26C0823039F4209701
:100D9000E1F084B5806284BDC8BD1DC0863041F4D9
:100DA0008091B00080688093B000C093B30013C0FE
:100DB000873041F48091B00080628093B000C0938E
:100DC000B40009C0C038D10514F460E001C061E08E
:100DD000812F0E940D07DF91CF911F910895282F39
:100DE00030E0C90185579F4FFC01949129583F4F2E
:100DF000F9018491882381F0E82FF0E0E859FF4F52
:100E0000E491F0E0662329F4808190958923808322
:100E100008958081892B80830895482F50E0CA016E
:100E200081569F4FFC012491CA0185579F4FFC01B9
:100E3000949149585F4FFA0134913323C1F1222331
:100E400031F1233021F4809180008F7705C0243068
:100E500031F4809180008F7D8093800018C0213014
:100E600019F484B58F7704C0223021F484B58F7DC6
:100E700084BD0DC0263021F48091B0008F7705C06D
:100E8000273029F48091B0008F7D8093B000E32F4C
:100E9000F0E0E359FF4FE491F0E0662329F480810C
:100EA00090958923808308958081892B808308957C
:100EB000EF92FF920F931F937B018C0122E030E0B1
:100EC00040E050E00E945A08205C3D4B404F5F4F8D
:100ED000CA01B901A80197010E945A08C901DA01A3
:100EE0000197A109B109292F3A2F4B2F552747FD0B
:100EF0005A950196A11DB11D2093C5008150809384
:100F0000C400E1ECF0E080818061808380818860B2
:100F100080838081806880831F910F91FF90EF9084
:100F20000895982F8091C00085FFFCCF9093C60054
:100F3000089580917D0190917E0180589F4F20916E
:100F40007F0130918001821B930B60E870E00E946A
:100F50002508089540917F015091800180917D0185
:100F600090917E018417950719F42FEF3FEF0FC082
:100F7000FA01EF57FE4F2081CA01019660E870E048
:100F80000E9425089093800180937F0130E0C90181
:100F900008951F920F920FB60F9211242F933F9333
:100FA0004F935F936F937F938F939F93AF93BF9371
:100FB000EF93FF934091C600E0917D01F0917E0197
:100FC000CF01019660E870E00E9425089C018091A5
:100FD0007F01909180012817390739F0EF57FE4FB4
:100FE000408330937E0120937D01FF91EF91BF916B
:100FF000AF919F918F917F916F915F914F913F91B1
:101000002F910F900FBE0F901F901895629FD001E7
:10101000739FF001829FE00DF11D649FE00DF11DB3
:10102000929FF00D839FF00D749FF00D659FF00D62
:101030009927729FB00DE11DF91F639FB00DE11D4F
:10104000F91FBD01CF011124089597FB092E072632
:101050000AD077FD04D049D006D000201AF470954C
:1010600061957F4F0895F6F7909581959F4F08956C
:10107000A1E21A2EAA1BBB1BFD010DC0AA1FBB1F9C
:10108000EE1FFF1FA217B307E407F50720F0A21B0E
:10109000B30BE40BF50B661F771F881F991F1A947B
:1010A00069F760957095809590959B01AC01BD01A5
:1010B000CF01089597FB092E05260ED057FD04D0C9
:1010C000D7DF0AD0001C38F4509540953095219513
:1010D0003F4F4F4F5F4F0895F6F79095809570956D
:1010E00061957F4F8F4F9F4F0895AA1BBB1B51E106
:1010F00007C0AA1FBB1FA617B70710F0A61BB70B88
:10110000881F991F5A95A9F780959095BC01CD012C
:101110000895EE0FFF1F0590F491E02D0994F894C7
:02112000FFCFFF
:10112200486F6C612C20736F7920656C20726F623E
:101132006F74206E756D65726F200006000B0008DB
:1011420000030001000200030009000A0001000080
:041152000000300465
:00000001FF
